:020000040000FA
:100000004EEF00F0B40EF66E000EF76E000EF86EB6
:100010000900F550056E0900F550066E055002E125
:1000200006503BE00900F550006E0900F550016EE6
:100030000900F550026E09000900F550E96E09004B
:10004000F550EA6E090009000900F550036E090039
:10005000F550046E09000900F6CF07F0F7CF08F05D
:10006000F8CF09F000C0F6FF01C0F7FF02C0F8FFAB
:10007000035002E1045007E00900F550EE6E03065C
:10008000F8E20406F9D707C0F6FF08C0F7FF09C079
:10009000F8FF0506C4E20606C5D7120017EEFFF00A
:1000A00027EEFFF0F86AA68EA69C02EC00F061EC49
:1000B00000F0FFD70100CE0000006000000001004A
:1000C000000093928A92E86AE86AFFD71200000063
:020000040030CA
:0E000000FFF2FFFEFFFFBBFFFFFFFFFFFFFF52
:00000001FF
